 Network

 Timestamp is 53c3c2e3 (Mon Jul 14 15:45:39 2014)

 Preferred load address is 0000000180000000

 Start         Length     Name                   Class
 0001:00000000 00000140H .idata$5                CODE
 0001:00000140 000006a2H .rdata                  CODE
 0001:000007f0 00008e2aH .text                   CODE
 0001:00009620 00000a6cH .xdata                  CODE
 0001:0000a08c 00000064H .idata$2                CODE
 0001:0000a0f0 00000014H .idata$3                CODE
 0001:0000a108 00000140H .idata$4                CODE
 0001:0000a248 000002a2H .idata$6                CODE
 0001:0000a4f0 00000182H .edata                  CODE
 0002:00000000 000001c0H .data                   DATA
 0002:000001c0 000010e0H .bss                    DATA
 0003:00000000 0000081cH .pdata                  DATA
 0004:00000000 00000058H .rsrc$01                DATA
 0004:00000060 00000370H .rsrc$02                DATA

  Address         Publics by Value              Rva+Base               Lib:Object

 0000:00000000       ___safe_se_handler_count   0000000000000000     <absolute>
 0000:00000000       ___safe_se_handler_table   0000000000000000     <absolute>
 0000:00000000       __ImageBase                0000000180000000     <linker-defined>
 0001:00000000       __imp_RegCloseKey          0000000180001000     advapi32:ADVAPI32.dll
 0001:00000008       __imp_RegOpenKeyExW        0000000180001008     advapi32:ADVAPI32.dll
 0001:00000010       \177ADVAPI32_NULL_THUNK_DATA 0000000180001010     advapi32:ADVAPI32.dll
 0001:00000018       __imp_ExpandEnvironmentStringsW 0000000180001018     kernel32:KERNEL32.dll
 0001:00000020       __imp_lstrcpyW             0000000180001020     kernel32:KERNEL32.dll
 0001:00000028       __imp_lstrlenW             0000000180001028     kernel32:KERNEL32.dll
 0001:00000030       __imp_lstrcmpiW            0000000180001030     kernel32:KERNEL32.dll
 0001:00000038       __imp_lstrcpynW            0000000180001038     kernel32:KERNEL32.dll
 0001:00000040       __imp_lstrcatW             0000000180001040     kernel32:KERNEL32.dll
 0001:00000048       __imp_GetModuleFileNameW   0000000180001048     kernel32:KERNEL32.dll
 0001:00000050       __imp_LocalFree            0000000180001050     kernel32:KERNEL32.dll
 0001:00000058       __imp_LocalAlloc           0000000180001058     kernel32:KERNEL32.dll
 0001:00000060       __imp_GetLogicalDrives     0000000180001060     kernel32:KERNEL32.dll
 0001:00000068       __imp_GetCurrentDirectoryW 0000000180001068     kernel32:KERNEL32.dll
 0001:00000070       __imp_lstrcmpW             0000000180001070     kernel32:KERNEL32.dll
 0001:00000078       __imp_SetLastError         0000000180001078     kernel32:KERNEL32.dll
 0001:00000080       __imp_FindClose            0000000180001080     kernel32:KERNEL32.dll
 0001:00000088       __imp_FindFirstFileW       0000000180001088     kernel32:KERNEL32.dll
 0001:00000090       __imp_GetComputerNameW     0000000180001090     kernel32:KERNEL32.dll
 0001:00000098       __imp_HeapAlloc            0000000180001098     kernel32:KERNEL32.dll
 0001:000000a0       __imp_HeapReAlloc          00000001800010a0     kernel32:KERNEL32.dll
 0001:000000a8       __imp_HeapFree             00000001800010a8     kernel32:KERNEL32.dll
 0001:000000b0       __imp_GetProcessHeap       00000001800010b0     kernel32:KERNEL32.dll
 0001:000000b8       __imp_GetSystemDirectoryW  00000001800010b8     kernel32:KERNEL32.dll
 0001:000000c0       __imp_GetLastError         00000001800010c0     kernel32:KERNEL32.dll
 0001:000000c8       __imp_SetCurrentDirectoryW 00000001800010c8     kernel32:KERNEL32.dll
 0001:000000d0       \177KERNEL32_NULL_THUNK_DATA 00000001800010d0     kernel32:KERNEL32.dll
 0001:000000d8       __imp_WNetCloseEnum        00000001800010d8     mpr:MPR.dll
 0001:000000e0       __imp_WNetOpenEnumW        00000001800010e0     mpr:MPR.dll
 0001:000000e8       __imp_WNetGetResourceInformationW 00000001800010e8     mpr:MPR.dll
 0001:000000f0       __imp_WNetGetResourceParentW 00000001800010f0     mpr:MPR.dll
 0001:000000f8       __imp_WNetAddConnection2W  00000001800010f8     mpr:MPR.dll
 0001:00000100       __imp_WNetCancelConnection2W 0000000180001100     mpr:MPR.dll
 0001:00000108       __imp_WNetEnumResourceW    0000000180001108     mpr:MPR.dll
 0001:00000110       \177MPR_NULL_THUNK_DATA    0000000180001110     mpr:MPR.dll
 0001:00000118       __imp_NetShareEnum         0000000180001118     Netapi32:NETAPI32.dll
 0001:00000120       __imp_NetApiBufferFree     0000000180001120     Netapi32:NETAPI32.dll
 0001:00000128       \177NETAPI32_NULL_THUNK_DATA 0000000180001128     Netapi32:NETAPI32.dll
 0001:00000130       __imp_CharUpperW           0000000180001130     user32:USER32.dll
 0001:00000138       \177USER32_NULL_THUNK_DATA 0000000180001138     user32:USER32.dll
 0001:00000140       MainGuid                   0000000180001140     Network.obj
 0001:00000150       MenuGuid                   0000000180001150     Network.obj
 0001:00000160       ConfigDialogGuid           0000000180001160     Network.obj
 0001:00000170       DisconnectDialogGuid       0000000180001170     Network.obj
 0001:00000180       UserPassDialogGuid         0000000180001180     Network.obj
 0001:00000190       ??_C@_1DE@BGKMIKPD@?$AAE?$AAu?$AAg?$AAe?$AAn?$AAe?$AA?5?$AAR?$AAo?$AAs?$AAh?$AAa?$AAl?$AA?5?$AA?$CG?$AA?5?$AAF?$AAa?$AAr?$AA?5?$AAG?$AAr?$AAo?$AAu?$AAp?$AA?$AA@ 0000000180001190     Network.obj
 0001:000001c8       ??_C@_1DO@KECGBOGC@?$AAN?$AAe?$AAt?$AAw?$AAo?$AAr?$AAk?$AA?5?$AAP?$AAl?$AAu?$AAg?$AAi?$AAn?$AA?5?$AAf?$AAo?$AAr?$AA?5?$AAF?$AAa?$AAr?$AA?5?$AAM?$AAa?$AAn?$AAa?$AAg?$AAe?$AAr?$AA?$AA@ 00000001800011c8     Network.obj
 0001:00000208       ??_C@_1BA@IFBJBPAK@?$AAN?$AAe?$AAt?$AAw?$AAo?$AAr?$AAk?$AA?$AA@ 0000000180001208     Network.obj
 0001:00000218       ??_C@_17ODNIDLDN@?$AAn?$AAe?$AAt?$AA?$AA@ 0000000180001218     Network.obj
 0001:00000220       ??_C@_19HNBCINPI@?$AAn?$AAe?$AAt?$AAg?$AA?$AA@ 0000000180001220     Network.obj
 0001:0000022c       ??_C@_15LEKKCGMK@?$AA?2?$AA?2?$AA?$AA@ 000000018000122c     Network.obj
 0001:00000238       ??_C@_1BE@OMHKNOGL@?$AAP?$AAa?$AAn?$AAe?$AAl?$AAM?$AAo?$AAd?$AAe?$AA?$AA@ 0000000180001238     NetCfg.obj
 0001:00000250       ??_C@_1CE@JCLLPGFN@?$AAN?$AAa?$AAv?$AAi?$AAg?$AAa?$AAt?$AAe?$AAT?$AAo?$AAD?$AAo?$AAm?$AAa?$AAi?$AAn?$AAs?$AA?$AA@ 0000000180001250     NetCfg.obj
 0001:00000278       ??_C@_1CE@DLMGFKCB@?$AAN?$AAo?$AAR?$AAo?$AAo?$AAt?$AAD?$AAo?$AAu?$AAb?$AAl?$AAe?$AAP?$AAo?$AAi?$AAn?$AAt?$AA?$AA@ 0000000180001278     NetCfg.obj
 0001:000002a0       ??_C@_1BO@LADGPGKF@?$AAF?$AAa?$AAv?$AAo?$AAr?$AAi?$AAt?$AAe?$AAs?$AAF?$AAl?$AAa?$AAg?$AAs?$AA?$AA@ 00000001800012a0     NetCfg.obj
 0001:000002c0       ??_C@_1BO@FLKJOEGH@?$AAF?$AAu?$AAl?$AAl?$AAP?$AAa?$AAt?$AAh?$AAS?$AAh?$AAa?$AAr?$AAe?$AAs?$AA?$AA@ 00000001800012c0     NetCfg.obj
 0001:000002e0       ??_C@_1CK@LKLAIIEF@?$AAH?$AAi?$AAd?$AAd?$AAe?$AAn?$AAS?$AAh?$AAa?$AAr?$AAe?$AAs?$AAA?$AAs?$AAH?$AAi?$AAd?$AAd?$AAe?$AAn?$AA?$AA@ 00000001800012e0     NetCfg.obj
 0001:00000310       ??_C@_1CC@DJEEMKIM@?$AAR?$AAe?$AAm?$AAo?$AAv?$AAe?$AAC?$AAo?$AAn?$AAn?$AAe?$AAc?$AAt?$AAi?$AAo?$AAn?$AA?$AA@ 0000000180001310     NetCfg.obj
 0001:00000338       ??_C@_1BO@ONNGHKLG@?$AAD?$AAi?$AAs?$AAc?$AAo?$AAn?$AAn?$AAe?$AAc?$AAt?$AAM?$AAo?$AAd?$AAe?$AA?$AA@ 0000000180001338     NetCfg.obj
 0001:00000358       ??_C@_1BK@IMMOFPGP@?$AAL?$AAo?$AAc?$AAa?$AAl?$AAN?$AAe?$AAt?$AAw?$AAo?$AAr?$AAk?$AA?$AA@ 0000000180001358     NetCfg.obj
 0001:00000378       ??_C@_1BK@BMPKBAI@?$AAS?$AAh?$AAo?$AAw?$AAP?$AAr?$AAi?$AAn?$AAt?$AAe?$AAr?$AAs?$AA?$AA@ 0000000180001378     NetCfg.obj
 0001:00000398       ??_C@_1BK@KLHOCBFH@?$AAH?$AAi?$AAd?$AAd?$AAe?$AAn?$AAS?$AAh?$AAa?$AAr?$AAe?$AAs?$AA?$AA@ 0000000180001398     NetCfg.obj
 0001:000003b8       ??_C@_1BC@ENICKDH@?$AAC?$AAo?$AAn?$AAt?$AAe?$AAn?$AAt?$AAs?$AA?$AA@ 00000001800013b8     NetCfg.obj
 0001:000003d0       ??_C@_1CC@PNNAOHJC@?$AAA?$AAd?$AAd?$AAT?$AAo?$AAP?$AAl?$AAu?$AAg?$AAi?$AAn?$AAs?$AAM?$AAe?$AAn?$AAu?$AA?$AA@ 00000001800013d0     NetCfg.obj
 0001:000003f8       ??_C@_1BO@NGDOFANC@?$AAA?$AAd?$AAd?$AAT?$AAo?$AAD?$AAi?$AAs?$AAk?$AAs?$AAM?$AAe?$AAn?$AAu?$AA?$AA@ 00000001800013f8     NetCfg.obj
 0001:00000418       ??_C@_1BC@EJKAECLA@?$AAn?$AAe?$AAt?$AA?3?$AAn?$AAe?$AAt?$AAg?$AA?$AA@ 0000000180001418     NetCfg.obj
 0001:00000430       ??_7?$DialogBuilderBase@UFarDialogItem@@@@6B@ 0000000180001430     NetCfg.obj
 0001:00000480       ??_7PluginDialogBuilder@@6B@ 0000000180001480     NetCfg.obj
 0001:000004c8       ??_7?$DialogItemBinding@UFarDialogItem@@@@6B@ 00000001800014c8     NetCfg.obj
 0001:000004d8       ??_7PluginCheckBoxBinding@@6B@ 00000001800014d8     NetCfg.obj
 0001:000004e8       ??_7PluginRadioButtonBinding@@6B@ 00000001800014e8     NetCfg.obj
 0001:000004f8       ??_C@_15EFLNJKHH@?$AA?$CF?$AAu?$AA?$AA@ 00000001800014f8     NetCfg.obj
 0001:00000500       ??_7PluginIntEditFieldBinding@@6B@ 0000000180001500     NetCfg.obj
 0001:00000510       ??_7PluginUIntEditFieldBinding@@6B@ 0000000180001510     NetCfg.obj
 0001:00000520       ??_C@_11LOCGONAA@?$AA?$AA@ 0000000180001520     NetCfg.obj
 0001:00000528       ??_C@_1O@BJPKKLLM@?$AAC?$AAo?$AAn?$AAf?$AAi?$AAg?$AA?$AA@ 0000000180001528     NetCfg.obj
 0001:00000548       ??_C@_13LBAGMAIH@?$AA?6?$AA?$AA@ 0000000180001548     NetClass.obj
 0001:00000550       ??_C@_1M@ICMPIFCG@?$AA0?$AA?0?$AA2?$AA?0?$AA0?$AA?$AA@ 0000000180001550     NetClass.obj
 0001:00000560       ??_C@_17DFFMIGIM@?$AA0?$AA?0?$AA2?$AA?$AA@ 0000000180001560     NetClass.obj
 0001:00000568       ??_C@_1BA@LKKFCKCJ@?$AAN?$AA?0?$AAC?$AA0?$AA?0?$AAC?$AA1?$AA?$AA@ 0000000180001568     NetClass.obj
 0001:00000578       ??_C@_19ELDIFHOA@?$AAN?$AA?0?$AAC?$AA0?$AA?$AA@ 0000000180001578     NetClass.obj
 0001:00000588       ??_C@_1BC@BDJLNJKB@?$AA?5?$AA?$CF?$AAs?$AA?3?$AA?5?$AA?$CF?$AAs?$AA?5?$AA?$AA@ 0000000180001588     NetClass.obj
 0001:000005a0       ??_C@_1BE@DEAPIJA@?$AAM?$AAi?$AAc?$AAr?$AAo?$AAs?$AAo?$AAf?$AAt?$AA?$AA@ 00000001800015a0     NetClass.obj
 0001:000005b8       ??_C@_19POFGONBN@?$AA?$CG?$AA?$CF?$AAc?$AA?3?$AA?$AA@ 00000001800015b8     NetClass.obj
 0001:000005c8       ??_C@_1M@JNLNDDIN@?$AA?$CF?$AAT?$AAM?$AAP?$AA?$CF?$AA?$AA@ 00000001800015c8     NetClass.obj
 0001:000005d4       ??_C@_15JNBOKNOG@?$AA?$AN?$AA?6?$AA?$AA@ 00000001800015d4     NetClass.obj
 0001:000005dc       ??_C@_13HOIJIPNN@?$AA?5?$AA?$AA@ 00000001800015dc     NetClass.obj
 0001:000005e0       ??_C@_15PCEAIKAA@?$AA?4?$AA?2?$AA?$AA@ 00000001800015e0     NetClass.obj
 0001:000005e8       ??_C@_15DDHGOCBH@?$AA?4?$AA?4?$AA?$AA@ 00000001800015e8     NetClass.obj
 0001:000005f0       ??_C@_19CDBNEOLI@?$AA?$CF?$AAs?$AA?2?$AA?$CK?$AA?$AA@ 00000001800015f0     NetClass.obj
 0001:00000600       ??_C@_1BI@HGBMBLHP@?$AA?2?$AA?2?$AA?$DP?$AA?2?$AAU?$AAN?$AAC?$AA?$CF?$AAs?$AA?2?$AA?$CK?$AA?$AA@ 0000000180001600     NetClass.obj
 0001:00000618       ??_C@_1BM@EONNLOAH@?$AAR?$AAe?$AAm?$AAo?$AAv?$AAe?$AAI?$AAt?$AAe?$AAm?$AAF?$AAa?$AAv?$AA?$AA@ 0000000180001618     NetClass.obj
 0001:00000638       ??_C@_1DA@CMNOOJGO@?$AAF?$AAa?$AAi?$AAl?$AAe?$AAd?$AA?5?$AAt?$AAo?$AA?5?$AAc?$AAr?$AAe?$AAa?$AAt?$AAe?$AA?5?$AAf?$AAo?$AAl?$AAd?$AAe?$AAr?$AA?$AA@ 0000000180001638     NetClass.obj
 0001:00000668       ??_C@_19INGAAIIO@?$AAI?$AAP?$AAC?$AA$?$AA?$AA@ 0000000180001668     NetClass.obj
 0001:00000674       ??_C@_13FPGAJAPJ@?$AA?2?$AA?$AA@ 0000000180001674     NetClass.obj
 0001:00000678       ??_7PluginEditFieldBinding@@6B@ 0000000180001678     NetClass.obj
 0001:00000688       ??_C@_1CC@FMHKFHHK@?$AAT?$AAh?$AAi?$AAs?$AA?5?$AAi?$AAs?$AA?5?$AAa?$AA?5?$AAd?$AAo?$AAm?$AAa?$AAi?$AAn?$AA?$AA@ 0000000180001688     NetClass.obj
 0001:000006b0       ??_C@_1CC@LMAEILBC@?$AAT?$AAh?$AAi?$AAs?$AA?5?$AAi?$AAs?$AA?5?$AAa?$AA?5?$AAS?$AAE?$AAR?$AAV?$AAE?$AAR?$AA?$AA@ 00000001800016b0     NetClass.obj
 0001:000006d8       ??_C@_19IEEMEPMH@?$AAD?$AAa?$AAt?$AAa?$AA?$AA@ 00000001800016d8     NetClass.obj
 0001:000006e8       ??_C@_1M@DFKENGJN@?$AA?$CF?$AAs?$AA?2?$AA?$CF?$AAs?$AA?$AA@ 00000001800016e8     NetClass.obj
 0001:000006f4       ??_C@_13EFKPHINO@?$AA?$EA?$AA?$AA@ 00000001800016f4     NetClass.obj
 0001:000006f8       ??_C@_13DMCFHHKM@?$AA3?$AA?$AA@ 00000001800016f8     NetClass.obj
 0001:00000700       ??_C@_1CA@FPAJCONG@?$AAD?$AAi?$AAs?$AAc?$AAo?$AAn?$AAn?$AAe?$AAc?$AAt?$AAD?$AAr?$AAi?$AAv?$AAe?$AA?$AA@ 0000000180001700     NetClass.obj
 0001:00000720       ??_C@_1BG@PFLPMIKK@?$AAN?$AAe?$AAt?$AAw?$AAo?$AAr?$AAk?$AA?2?$AA?$CF?$AAc?$AA?$AA@ 0000000180001720     NetClass.obj
 0001:00000738       ??_C@_1BI@LJGELBNP@?$AAN?$AAe?$AAt?$AAw?$AAo?$AAr?$AAk?$AAU?$AAs?$AAe?$AAr?$AA?$AA@ 0000000180001738     NetClass.obj
 0001:00000750       ??_C@_13GGAHEHIG@?$AA?$AB?$AA?$AA@ 0000000180001750     NetClass.obj
 0001:00000758       ??_C@_1BI@PJIFJHLI@?$AAM?$AAa?$AAk?$AAe?$AA?5?$AAF?$AAo?$AAl?$AAd?$AAe?$AAr?$AA?$AA@ 0000000180001758     NetCommon.obj
 0001:00000770       ??_C@_1BK@LDEGEPBC@?$AAF?$AAo?$AAl?$AAd?$AAe?$AAr?$AA?5?$AAn?$AAa?$AAm?$AAe?$AA?3?$AA?$AA@ 0000000180001770     NetCommon.obj
 0001:00000790       ??_C@_1BE@BIEMJOKH@?$AAN?$AAe?$AAw?$AAF?$AAo?$AAl?$AAd?$AAe?$AAr?$AA?$AA@ 0000000180001790     NetCommon.obj
 0001:000007a4       ??_C@_15MNCACJLI@?$AA?2?$AA?1?$AA?$AA@ 00000001800017a4     NetFavorites.obj
 0001:000007b0       ??_C@_1BE@PDPMPIAC@?$AAF?$AAa?$AAv?$AAo?$AAr?$AAi?$AAt?$AAe?$AAs?$AA?$AA@ 00000001800017b0     NetFavorites.obj
 0001:000007c8       ??_C@_1BK@GCNMKDHP@?$AAF?$AAa?$AAv?$AAo?$AAr?$AAi?$AAt?$AAe?$AAs?$AA?2?$AA?$CF?$AAs?$AA?$AA@ 00000001800017c8     NetFavorites.obj
 0001:00000800       __chkstk                   0000000180001800 f   chkstk.obj
 0001:00000800       _alloca_probe              0000000180001800     chkstk.obj
 0001:00000850       GetGlobalInfoW             0000000180001850 f   Network.obj
 0001:000008d0       ClosePanelW                00000001800018d0 f   Network.obj
 0001:00000900       GetFindDataW               0000000180001900 f   Network.obj
 0001:00000920       FreeFindDataW              0000000180001920 f   Network.obj
 0001:00000940       GetOpenPanelInfoW          0000000180001940 f   Network.obj
 0001:00000950       SetDirectoryW              0000000180001950 f   Network.obj
 0001:00000970       DeleteFilesW               0000000180001970 f   Network.obj
 0001:00000990       ProcessPanelInputW         0000000180001990 f   Network.obj
 0001:000009b0       ProcessPanelEventW         00000001800019b0 f   Network.obj
 0001:000009d0       OpenW                      00000001800019d0 f   Network.obj
 0001:00000c60       ?GetLangString@PluginDialogBuilder@@MEAAPEB_WH@Z 0000000180001c60 f i NetCfg.obj
 0001:00000c70       GetPluginInfoW             0000000180001c70 f   NetCfg.obj
 0001:00000d20       ?InitDialogItem@?$DialogBuilderBase@UFarDialogItem@@@@MEAAXPEAUFarDialogItem@@PEB_W@Z 0000000180001d20 f i NetCfg.obj
 0001:00000d20       ?WriteFavoriteItem@@YAXPEAU_FAVORITEITEM@@PEA_W@Z 0000000180001d20 f i NetFavorites.obj
 0001:00000d20       ?SaveValue@?$DialogItemBinding@UFarDialogItem@@@@UEAAXPEAUFarDialogItem@@H@Z 0000000180001d20 f i NetCfg.obj
 0001:00000d30       ?TextWidth@?$DialogBuilderBase@UFarDialogItem@@@@MEAAHAEBUFarDialogItem@@@Z 0000000180001d30 f i NetCfg.obj
 0001:00000d40       ?DoShowDialog@?$DialogBuilderBase@UFarDialogItem@@@@MEAA_JXZ 0000000180001d40 f i NetCfg.obj
 0001:00000d50       ??1?$DialogBuilderBase@UFarDialogItem@@@@MEAA@XZ 0000000180001d50 f i NetCfg.obj
 0001:00000dd0       ??_E?$DialogBuilderBase@UFarDialogItem@@@@MEAAPEAXI@Z 0000000180001dd0 f i NetCfg.obj
 0001:00000dd0       ??_G?$DialogBuilderBase@UFarDialogItem@@@@MEAAPEAXI@Z 0000000180001dd0 f i NetCfg.obj
 0001:00000e00       ?ReallocDialogItems@?$DialogBuilderBase@UFarDialogItem@@@@IEAAXXZ 0000000180001e00 f i NetCfg.obj
 0001:00000f20       ?MaxTextWidth@?$DialogBuilderBase@UFarDialogItem@@@@IEAA_JXZ 0000000180001f20 f i NetCfg.obj
 0001:00001040       ?InitDialogItem@PluginDialogBuilder@@MEAAXPEAUFarDialogItem@@PEB_W@Z 0000000180002040 f i NetCfg.obj
 0001:00001070       ?TextWidth@PluginDialogBuilder@@MEAAHAEBUFarDialogItem@@@Z 0000000180002070 f i NetCfg.obj
 0001:00001080       ?DoShowDialog@PluginDialogBuilder@@MEAA_JXZ 0000000180002080 f i NetCfg.obj
 0001:00001120       ?SaveValue@PluginCheckBoxBinding@@UEAAXPEAUFarDialogItem@@H@Z 0000000180002120 f i NetCfg.obj
 0001:00001180       ?SaveValue@PluginRadioButtonBinding@@UEAAXPEAUFarDialogItem@@H@Z 0000000180002180 f i NetCfg.obj
 0001:000011d0       ??0PluginIntEditFieldBinding@@QEAA@AEBUPluginStartupInfo@@PEAPEAXHPEAHH@Z 00000001800021d0 f i NetCfg.obj
 0001:00001290       ?SaveValue@PluginIntEditFieldBinding@@UEAAXPEAUFarDialogItem@@H@Z 0000000180002290 f i NetCfg.obj
 0001:000012e0       ??0PluginUIntEditFieldBinding@@QEAA@AEBUPluginStartupInfo@@PEAPEAXHPEAIH@Z 00000001800022e0 f i NetCfg.obj
 0001:000013a0       ?SaveValue@PluginUIntEditFieldBinding@@UEAAXPEAUFarDialogItem@@H@Z 00000001800023a0 f i NetCfg.obj
 0001:000013f0       ?CreateCheckBoxBinding@PluginDialogBuilder@@MEAAPEAU?$DialogItemBinding@UFarDialogItem@@@@PEAHH@Z 00000001800023f0 f i NetCfg.obj
 0001:00001470       ?CreateRadioButtonBinding@PluginDialogBuilder@@MEAAPEAU?$DialogItemBinding@UFarDialogItem@@@@PEAH@Z 0000000180002470 f i NetCfg.obj
 0001:000014e0       ??_GPluginDialogBuilder@@UEAAPEAXI@Z 00000001800024e0 f i NetCfg.obj
 0001:000014e0       ??_EPluginDialogBuilder@@UEAAPEAXI@Z 00000001800024e0 f i NetCfg.obj
 0001:00001530       ?UpdateBorderSize@?$DialogBuilderBase@UFarDialogItem@@@@IEAAXXZ 0000000180002530 f i NetCfg.obj
 0001:000015f0       ??_GPluginIntEditFieldBinding@@UEAAPEAXI@Z 00000001800025f0 f i NetCfg.obj
 0001:000015f0       ??_GPluginEditFieldBinding@@UEAAPEAXI@Z 00000001800025f0 f i NetClass.obj
 0001:000015f0       ??_EPluginIntEditFieldBinding@@UEAAPEAXI@Z 00000001800025f0 f i NetCfg.obj
 0001:000015f0       ??_EPluginEditFieldBinding@@UEAAPEAXI@Z 00000001800025f0 f i NetClass.obj
 0001:000015f0       ??_GPluginCheckBoxBinding@@UEAAPEAXI@Z 00000001800025f0 f i NetCfg.obj
 0001:000015f0       ??_EPluginUIntEditFieldBinding@@UEAAPEAXI@Z 00000001800025f0 f i NetCfg.obj
 0001:000015f0       ??_EPluginCheckBoxBinding@@UEAAPEAXI@Z 00000001800025f0 f i NetCfg.obj
 0001:000015f0       ??_GPluginUIntEditFieldBinding@@UEAAPEAXI@Z 00000001800025f0 f i NetCfg.obj
 0001:000015f0       ??_E?$DialogItemBinding@UFarDialogItem@@@@UEAAPEAXI@Z 00000001800025f0 f i NetCfg.obj
 0001:000015f0       ??_G?$DialogItemBinding@UFarDialogItem@@@@UEAAPEAXI@Z 00000001800025f0 f i NetCfg.obj
 0001:000015f0       ??_EPluginRadioButtonBinding@@UEAAPEAXI@Z 00000001800025f0 f i NetCfg.obj
 0001:000015f0       ??_GPluginRadioButtonBinding@@UEAAPEAXI@Z 00000001800025f0 f i NetCfg.obj
 0001:00001620       ?AddIntEditField@PluginDialogBuilder@@UEAAPEAUFarDialogItem@@PEAHH@Z 0000000180002620 f i NetCfg.obj
 0001:00001730       ?AddUIntEditField@PluginDialogBuilder@@UEAAPEAUFarDialogItem@@PEAIH@Z 0000000180002730 f i NetCfg.obj
 0001:00001840       ?Config@@YAHXZ             0000000180002840 f   NetCfg.obj
 0001:00002c80       ?Alloc@SimpleString@@AEAAX_K@Z 0000000180003c80 f i NetClass.obj
 0001:00002cf0       ??0SimpleString@@QEAA@PEB_W_K@Z 0000000180003cf0 f i NetClass.obj
 0001:00002da0       ?Inflate@SimpleString@@QEAAX_K@Z 0000000180003da0 f i NetClass.obj
 0001:00002ed0       ??0NetResourceList@@QEAA@XZ 0000000180003ed0 f   NetClass.obj
 0001:00002ee0       ?InitNetResource@NetResourceList@@SAXAEAU_NETRESOURCEW@@@Z 0000000180003ee0 f   NetClass.obj
 0001:00002f00       ?CopyNetResource@NetResourceList@@SAXAEAU_NETRESOURCEW@@AEBU2@@Z 0000000180003f00 f   NetClass.obj
 0001:00002fe0       ?Push@NetResourceList@@QEAAXAEAU_NETRESOURCEW@@@Z 0000000180003fe0 f   NetClass.obj
 0001:00003060       ?Pop@NetResourceList@@QEAAXXZ 0000000180004060 f   NetClass.obj
 0001:000030d0       ?GotoFavorite@NetBrowser@@QEAAHPEA_W@Z 00000001800040d0 f   NetClass.obj
 0001:00003190       ?FreeFindData@NetBrowser@@QEAAXPEAUPluginPanelItem@@H@Z 0000000180004190 f   NetClass.obj
 0001:00003210       ?GetDriveToDisconnect@NetBrowser@@AEAAHPEB_WPEA_W@Z 0000000180004210 f   NetClass.obj
 0001:000033c0       ?GetOpenPanelInfo@NetBrowser@@QEAAXPEAUOpenPanelInfo@@@Z 00000001800043c0 f   NetClass.obj
 0001:000036c0       ?IsMSNetResource@NetBrowser@@SAHAEBU_NETRESOURCEW@@@Z 00000001800046c0 f   NetClass.obj
 0001:00003700       ?GetResourceInfo@NetBrowser@@SAHPEA_WPEAU_NETRESOURCEW@@@Z 0000000180004700 f   NetClass.obj
 0001:00003800       ?GetResourceParent@NetBrowser@@SAHAEAU_NETRESOURCEW@@PEAU2@@Z 0000000180004800 f   NetClass.obj
 0001:00003990       ?AskMapDrive@NetBrowser@@AEAAHPEA_WAEAH@Z 0000000180004990 f   NetClass.obj
 0001:00003ba0       ?DisconnectFromServer@NetBrowser@@CAXPEAU_NETRESOURCEW@@@Z 0000000180004ba0 f   NetClass.obj
 0001:00003df0       ?GetLocalName@NetBrowser@@AEAAXPEA_W0@Z 0000000180004df0 f   NetClass.obj
 0001:00003ee0       ?FileNames2Clipboard@NetBrowser@@AEAAXH@Z 0000000180004ee0 f   NetClass.obj
 0001:000041d0       ?GetRemoteName@NetBrowser@@AEAAXPEAU_NETRESOURCEW@@PEA_W@Z 00000001800051d0 f   NetClass.obj
 0001:00004290       ?IsReadable@NetBrowser@@AEAAHPEB_W@Z 0000000180005290 f   NetClass.obj
 0001:00004340       ?SetOpenFromCommandLine@NetBrowser@@QEAAXPEA_W@Z 0000000180005340 f   NetClass.obj
 0001:00004350       ?SetOpenFromFilePanel@NetBrowser@@QEAAHPEA_W@Z 0000000180005350 f   NetClass.obj
 0001:000043d0       ?GotoLocalNetwork@NetBrowser@@QEAAXXZ 00000001800053d0 f   NetClass.obj
 0001:00004530       ?SetCursorToShare@NetBrowser@@AEAAXPEA_W@Z 0000000180005530 f   NetClass.obj
 0001:000046c0       ?RemoveItems@NetBrowser@@AEAAXXZ 00000001800056c0 f   NetClass.obj
 0001:000049a0       ?CreateFavSubFolder@NetBrowser@@QEAAXXZ 00000001800059a0 f   NetClass.obj
 0001:00004a60       ?GetHiddenShares@NetBrowser@@AEAAXXZ 0000000180005a60 f   NetClass.obj
 0001:00004d60       ?SaveValue@PluginEditFieldBinding@@UEAAXPEAUFarDialogItem@@H@Z 0000000180005d60 f i NetClass.obj
 0001:00004da0       ?Replace@SimpleString@@QEAAAEAV1@_K0PEB_W0@Z 0000000180005da0 f i NetClass.obj
 0001:00004f20       ?Clear@NetResourceList@@QEAAXXZ 0000000180005f20 f   NetClass.obj
 0001:00004fb0       ?Enumerate@NetResourceList@@QEAAHKKKPEAU_NETRESOURCEW@@@Z 0000000180005fb0 f   NetClass.obj
 0001:00005160       ?EnumerateNetList@NetBrowser@@AEAAHXZ 0000000180006160 f   NetClass.obj
 0001:00005350       ?IsResourceReadable@NetBrowser@@SAHAEAU_NETRESOURCEW@@@Z 0000000180006350 f   NetClass.obj
 0001:00005430       ?EditFavorites@NetBrowser@@QEAAHXZ 0000000180006430 f   NetClass.obj
 0001:00005760       ?AddConnectionWithLogon@NetBrowser@@SAHPEAU_NETRESOURCEW@@PEA_W1H@Z 0000000180006760 f   NetClass.obj
 0001:000058f0       ?AddConnectionFromFavorites@NetBrowser@@SAHPEAU_NETRESOURCEW@@H@Z 00000001800068f0 f   NetClass.obj
 0001:000059a0       ??4NetResourceList@@QEAAAEAV0@AEAV0@@Z 00000001800069a0 f   NetClass.obj
 0001:00005a60       ??0NetBrowser@@QEAA@XZ     0000000180006a60 f   NetClass.obj
 0001:00005c30       ??1NetBrowser@@QEAA@XZ     0000000180006c30 f   NetClass.obj
 0001:00005c60       ?ProcessEvent@NetBrowser@@QEAAH_JPEAX@Z 0000000180006c60 f   NetClass.obj
 0001:00005e20       ExitFARW                   0000000180006e20 f   NetClass.obj
 0001:00005e80       ?ConfirmCancelConnection@NetBrowser@@AEAAHPEA_W0AEAH@Z 0000000180006e80 f   NetClass.obj
 0001:00006740       ?GetNameAndPassword@NetBrowser@@CAHPEAU__NameAndPassInfo@@@Z 0000000180007740 f   NetClass.obj
 0001:00007130       ?CancelConnection@NetBrowser@@AEAAHPEB_W@Z 0000000180008130 f   NetClass.obj
 0001:000073e0       ?AddConnectionExplicit@NetBrowser@@SAHPEAU_NETRESOURCEW@@H@Z 00000001800083e0 f   NetClass.obj
 0001:000074f0       ?GotoComputer@NetBrowser@@AEAAHPEB_W@Z 00000001800084f0 f   NetClass.obj
 0001:00007720       ?GetFindData@NetBrowser@@QEAAHPEAPEAUPluginPanelItem@@PEA_K_K@Z 0000000180008720 f   NetClass.obj
 0001:00007a90       ?DeleteFiles@NetBrowser@@QEAAHPEAUPluginPanelItem@@H_K@Z 0000000180008a90 f   NetClass.obj
 0001:00007b40       ?ChangeToDirectory@NetBrowser@@AEAAHPEB_WHH@Z 0000000180008b40 f   NetClass.obj
 0001:00008060       ?MapNetworkDrive@NetBrowser@@AEAAHPEB_WHH@Z 0000000180009060 f   NetClass.obj
 0001:00008470       ?SetDirectory@NetBrowser@@QEAAHPEB_W_K@Z 0000000180009470 f   NetClass.obj
 0001:00008710       ?ProcessKey@NetBrowser@@QEAAHPEBU_INPUT_RECORD@@@Z 0000000180009710 f   NetClass.obj
 0001:00008b70       SetStartupInfoW            0000000180009b70 f   NetCommon.obj
 0001:00008f90       ConfigureW                 0000000180009f90 f   NetCommon.obj
 0001:00008fa0       ?DlgCreateFolder@@YAHPEA_WH@Z 0000000180009fa0 f   NetCommon.obj
 0001:00009000       ?GetFavorites@@YAHPEAU_NETRESOURCEW@@PEAVNetResourceList@@@Z 000000018000a000 f   NetFavorites.obj
 0001:000090e0       ?CheckFavoriteItem@@YAHQEAU_NETRESOURCEW@@@Z 000000018000a0e0 f   NetFavorites.obj
 0001:00009110       ?GetFavoritesParent@@YAHAEAU_NETRESOURCEW@@PEAU1@@Z 000000018000a110 f   NetFavorites.obj
 0001:000091f0       ?AddUIntEditField@?$DialogBuilderBase@UFarDialogItem@@@@UEAAPEAUFarDialogItem@@PEAIH@Z 000000018000a1f0 f   NetCfg.obj
 0001:000091f0       ?AddIntEditField@?$DialogBuilderBase@UFarDialogItem@@@@UEAAPEAUFarDialogItem@@PEAHH@Z 000000018000a1f0 f   NetCfg.obj
 0001:000091f0       ?ReadFavoriteItem@@YAHPEAU_FAVORITEITEM@@@Z 000000018000a1f0 f   NetFavorites.obj
 0001:000091f0       ?RemoveFromFavorites@@YAHPEA_WP6AK0PEAX@Z1@Z 000000018000a1f0 f   NetFavorites.obj
 0001:000091f0       ?GetFavoriteResource@@YAHPEB_WPEAU_NETRESOURCEW@@@Z 000000018000a1f0 f   NetFavorites.obj
 0001:000091f0       ?GetLangString@?$DialogBuilderBase@UFarDialogItem@@@@MEAAPEB_WH@Z 000000018000a1f0 f   NetCfg.obj
 0001:000091f0       ?CreateRadioButtonBinding@?$DialogBuilderBase@UFarDialogItem@@@@MEAAPEAU?$DialogItemBinding@UFarDialogItem@@@@PEAH@Z 000000018000a1f0 f   NetCfg.obj
 0001:000091f0       ?CreateCheckBoxBinding@?$DialogBuilderBase@UFarDialogItem@@@@MEAAPEAU?$DialogItemBinding@UFarDialogItem@@@@PEAHH@Z 000000018000a1f0 f   NetCfg.obj
 0001:000091f0       ?CreateSubFolder@@YAHPEA_W0@Z 000000018000a1f0 f   NetFavorites.obj
 0001:00009200       ?GetMsg@@YAPEB_WH@Z        000000018000a200 f   NetMix.obj
 0001:00009220       ??0TSaveScreen@@QEAA@XZ    000000018000a220 f   NetMix.obj
 0001:000092b0       ??1TSaveScreen@@QEAA@XZ    000000018000a2b0 f   NetMix.obj
 0001:000092e0       wcschr                     000000018000a2e0 f   libCRT64:strchr.obj
 0001:00009300       ??3@YAXPEAX@Z              000000018000a300 f   libCRT64:delete.obj
 0001:00009310       ??2@YAPEAX_K@Z             000000018000a310 f   libCRT64:new.obj
 0001:00009320       memset                     000000018000a320 f   libCRT64:memset.obj
 0001:00009350       ??_V@YAXPEAX@Z             000000018000a350 f   libCRT64:delete_array.obj
 0001:00009360       ??_U@YAPEAX_K@Z            000000018000a360 f   libCRT64:new_array.obj
 0001:00009370       memcpy                     000000018000a370 f   libCRT64:memcpy.obj
 0001:000093a0       wcsstr                     000000018000a3a0 f   libCRT64:strstr.obj
 0001:00009410       memmove                    000000018000a410 f   libCRT64:memmove.obj
 0001:00009470       realloc                    000000018000a470 f   libCRT64:realloc.obj
 0001:00009500       free                       000000018000a500 f   libCRT64:free.obj
 0001:00009530       wcsdup                     000000018000a530 f   libCRT64:strdup.obj
 0001:00009580       malloc                     000000018000a580 f   libCRT64:malloc.obj
 0001:000095b0       wcsncmp                    000000018000a5b0 f   libCRT64:strncmp.obj
 0001:000095e4       WNetGetResourceInformationW 000000018000a5e4 f   mpr:MPR.dll
 0001:000095ea       WNetGetResourceParentW     000000018000a5ea f   mpr:MPR.dll
 0001:000095f0       WNetAddConnection2W        000000018000a5f0 f   mpr:MPR.dll
 0001:000095f6       WNetCancelConnection2W     000000018000a5f6 f   mpr:MPR.dll
 0001:000095fc       WNetCloseEnum              000000018000a5fc f   mpr:MPR.dll
 0001:00009602       WNetEnumResourceW          000000018000a602 f   mpr:MPR.dll
 0001:00009608       WNetOpenEnumW              000000018000a608 f   mpr:MPR.dll
 0001:0000960e       NetApiBufferFree           000000018000a60e f   Netapi32:NETAPI32.dll
 0001:00009614       NetShareEnum               000000018000a614 f   Netapi32:NETAPI32.dll
 0001:0000a08c       __IMPORT_DESCRIPTOR_KERNEL32 000000018000b08c     kernel32:KERNEL32.dll
 0001:0000a0a0       __IMPORT_DESCRIPTOR_USER32 000000018000b0a0     user32:USER32.dll
 0001:0000a0b4       __IMPORT_DESCRIPTOR_ADVAPI32 000000018000b0b4     advapi32:ADVAPI32.dll
 0001:0000a0c8       __IMPORT_DESCRIPTOR_MPR    000000018000b0c8     mpr:MPR.dll
 0001:0000a0dc       __IMPORT_DESCRIPTOR_NETAPI32 000000018000b0dc     Netapi32:NETAPI32.dll
 0001:0000a0f0       __NULL_IMPORT_DESCRIPTOR   000000018000b0f0     kernel32:KERNEL32.dll
 0002:00000000       ?StrAddToDisksMenu@@3PEB_WEB 000000018000c000     NetCfg.obj
 0002:00000008       ?StrAddToPluginsMenu@@3PEB_WEB 000000018000c008     NetCfg.obj
 0002:00000010       ?StrHelpNetBrowse@@3PEB_WEB 000000018000c010     NetCfg.obj
 0002:00000018       ?StrHiddenShares@@3PEB_WEB 000000018000c018     NetCfg.obj
 0002:00000020       ?StrShowPrinters@@3PEB_WEB 000000018000c020     NetCfg.obj
 0002:00000028       ?StrLocalNetwork@@3PEB_WEB 000000018000c028     NetCfg.obj
 0002:00000030       ?StrDisconnectMode@@3PEB_WEB 000000018000c030     NetCfg.obj
 0002:00000038       ?StrRemoveConnection@@3PEB_WEB 000000018000c038     NetCfg.obj
 0002:00000040       ?StrHiddenSharesAsHidden@@3PEB_WEB 000000018000c040     NetCfg.obj
 0002:00000048       ?StrFullPathShares@@3PEB_WEB 000000018000c048     NetCfg.obj
 0002:00000050       ?StrFavoritesFlags@@3PEB_WEB 000000018000c050     NetCfg.obj
 0002:00000058       ?StrNoRootDoublePoint@@3PEB_WEB 000000018000c058     NetCfg.obj
 0002:00000060       ?StrNavigateToDomains@@3PEB_WEB 000000018000c060     NetCfg.obj
 0002:00000068       ?StrPanelMode@@3PEB_WEB    000000018000c068     NetCfg.obj
 0002:00000184       ?IsFirstRun@@3HA           000000018000c184     NetCommon.obj
 0002:00000188       ?szFavProv@@3PA_WA         000000018000c188     NetFavorites.obj
 0002:000001b8       ?g_szInvalidChars@@3PEB_WEB 000000018000c1b8     NetFavorites.obj
 0002:000001d0       ?CommonRootResources@@3PEAVNetResourceList@@EA 000000018000c1d0     NetClass.obj
 0002:000001d8       ?SavedCommonRootResources@@3HA 000000018000c1d8     NetClass.obj
 0002:00000fb0       ?CommonCurResource@@3U_NETRESOURCEW@@A 000000018000cfb0     NetCommon.obj
 0002:00000fe0       ?Info@@3UPluginStartupInfo@@A 000000018000cfe0     NetCommon.obj
 0002:000010f0       ?FSF@@3UFarStandardFunctions@@A 000000018000d0f0     NetCommon.obj
 0002:00001268       ?Opt@@3UOptions@@A         000000018000d268     NetCommon.obj
 0002:00001298       ?PCommonCurResource@@3PEAU_NETRESOURCEW@@EA 000000018000d298     NetCommon.obj

 entry point at        0000:00000000

 Static symbols

 0001:00002df0       ?GetSetting@@YA_JW4FARSETTINGS_SUBFOLDERS@@PEB_W@Z 0000000180003df0 f   NetClass.obj
